:020000040000FA
:040000008A015F28EA
:08000800CF308100A2011F1B93
:1000100022140130A002031CA10203183C28003066
:10002000A0000530A100AC1F1A28AB09AC09AB0F2A
:100030001A28AC0AAE1F2128AD09AE09AD0F212840
:10004000AE0A06102B08AF002C08B0002D08AF0731
:100050000318B00A2E08B0070030AF020318332887
:10006000B003B01B38280430B002B01B3828061487
:10007000AB01AC01AD01AE0122082406031D4428EA
:10008000AB0F4828AC0A48280130AB02031CAC0374
:1000900022082506031D5028AD0F5428AE0A542807
:1000A0000130AD02031CAE03A401A501A30A231B6A
:1000B0002414A31A25142408A5060B110900831281
:1000C000031385018601831603138B012B308500F2
:1000D000003086008312031314309F000516CF30C2
:1000E00081000030A0000530A100A3018316031396
:1000F00088308100A0308B008312031398137F286F
:02400E00421F4F
:00000001FF
